:020000040800F2
:10000000700400209D010008A50100085911000896
:10001000A9010008AB010008AD01000800000000C4
:10002000000000000000000000000000AF01000818
:10003000B101000800000000B301000871150008BC
:10004000B7010008B7010008B7010008B7010008B0
:10005000B7010008B7010008B7010008B7010008A0
:10006000B7010008B7010008B7010008B701000890
:10007000B7010008B7010008B7010008B701000880
:10008000B7010008B701000871080008B7010008AF
:100090007D090008B7010008B7010008B701000892
:1000A000B70100087D170008B7010008B701000874
:1000B000B7010008B7010008B7010008B701000840
:1000C000B7010008B7010008B7010008B701000830
:1000D000B70100080D180008B7010008B7010008B3
:1000E000B7010008B7010008B7010008B701000810
:1000F000B7010008B7010008B7010008B701000800
:10010000B7010008B7010008B7010008B7010008EF
:10011000C1170008B7010008B7010008B7010008BF
:10012000B7010008B7010008B7010008B7010008CF
:10013000B7010008B7010008B7010008B7010008BF
:10014000B7010008B7010008B7010008B7010008AF
:10015000B7010008B7010008B7010008B70100089F
:10016000B7010008B7010008B7010008B70100088F
:10017000B7010008B7010008B7010008B70100087F
:10018000B7010008B7010008DFF80CD000F0CCFA86
:1001900000480047192100087004002006488047E5
:1001A00006480047FEE7FEE7FEE7FEE7FEE7FEE75C
:1001B000FEE7FEE7FEE7FEE72117000889010008D9
:1001C00040EA01039B0703D009E008C9121F08C0D9
:1001D000042AFAD203E011F8013B00F8013B521E59
:1001E000F9D270472DE9FE4F804681EA0300C00F27
:1001F0000C46009021F0004123F00045B8EB0200CE
:10020000A94105D24046214690461C460B4602466F
:1002100023F00040104347D0270DC7F30A00C3F373
:100220000A510290401A019040286BDAC3F3130080
:1002300040F4801B0098924620B10023D2EB030AC1
:1002400063EB0B0B01985946C0F14002504600F099
:100250008DF906460D4650465946019A00F095F92B
:1002600010EB08006141002487EA115284EAE77329
:100270001A4340D0009A62B3019A012A4FEA07520A
:1002800015DC001B61EB02014FF0004202EA07524D
:10029000CDE90042001C41F5801132462B4600F0AA
:1002A000CCF903B0BDE8F08F40462146F9E7001BCA
:1002B00061EB0201001C41F5801300185B4120181E
:1002C000A2F5001747EB030140EAD570B6196D415E
:1002D00011E06D084FEA360645EAC0754FEA07524D
:1002E000001B61EB0201001C41F5801149084FEA37
:1002F00030000019514132462B4603B0BDE8F04FA3
:1003000000F08CB90098012240000023D0EB0202DB
:1003100063EBE073009821464FEAE074B8EB00000D
:1003200061EB0401E9E783F000435BE781F0004102
:1003300058E72DE9FE4F81EA030404F0004421F060
:10034000004100944FF0000B23F0004350EA0104F9
:100350005ED052EA03045BD0C3F30A54C1F30A55DA
:100360002C44A4F2F3340194A0FB0254C1F3130112
:1003700041F48011C3F3130343F4801301FB0244DF
:1003800000FB034E840A970A44EA815447EA8357E4
:10039000A4FB076802958D0A05FB07854FEA932C9D
:1003A00004FB0C542705029D4FEA065847EA16370E
:1003B000B5EB08056EEB070C870E920E47EA811726
:1003C00042EA8312A7FB0201B6EB0B0164EB0004C7
:1003D0002B0D43EA0C335E1844EB1C50DA465146B1
:1003E000E7FB0201C5F313044FEA0B3343EA14534E
:1003F0004FEA0432019C43EA0603A4F10C04029480
:10040000009CCDE900B400F018F903B0BDE8F08F0E
:1004100000200146F9E72DE9F04D81EA030404F0DC
:10042000004B21F0004514464FF0000A23F0004134
:1004300050EA050220D054EA01021DD0C5F30A5744
:100440000246C5F31303C1F31300C1F30A5640F487
:10045000801543F48013A7EB0608101BD64608F25C
:10046000FD3873EB050002D308F1010801E0921892
:100470005B41B8F1000F03DA00200146BDE8F08DC2
:1004800000204FF48011064684460EE0171B73EBE4
:10049000050705D3121B63EB050306434CEA010C69
:1004A00049084FEA300092185B4150EA0107EDD14C
:1004B00052EA030012D082EA040083EA05010843ED
:1004C00005D0101BAB4106D20122002306E000221A
:1004D0004FF0004302E06FF0010253101AEB0600E8
:1004E0004CEB085110EB0A0041EB0B01BDE8F04D5D
:1004F00000F094B80EB540F2334102910021CDE9ED
:1005000000110A460B4600F098F803B000BD00F059
:10051000004230F000400AD0C10D01F56071C0F317
:10052000160042EA0151C2084007114370470020FB
:100530000146704701F0004330B421F0004150EA19
:10054000010206D00A0DA2F56072C1F31301002A60
:1005500002DC30BC00207047440F44EAC104C100F3
:10056000E01830BC00EBC25000F021B8202A04DBB8
:10057000203A00FA02F1002070479140C2F12003B6
:1005800020FA03F3194390407047202A06DBCB176B
:10059000203A41FA02F043EAE07306E041FA02F33E
:1005A000D040C2F12002914008431946704700290B
:1005B000A8BF7047401C490008BF20F001007047E9
:1005C00010B4B0FA80FC00FA0CF050EA010404BF49
:1005D00010BC704749B1CCF1200421FA04F411FA9F
:1005E0000CF118BF012121430843A3EB0C01CB1DE3
:1005F0004FEA00614FEA102042BF002010BC704754
:1006000000EBC35010440029A4BF10BC7047401C2D
:10061000490008BF20F0010010BC704710B5141E3F
:1006200073F1000408DA401C41F1000192185B41AB
:100630001A4301D120F0010010BD2DE9F04D924682
:100640009B4611B1B1FA81F202E0B0FA80F2203299
:100650009046FFF78BFF04460F4640EA0A0041EA46
:100660000B0153465A46084313D0114653EA010082
:1006700019D0C8F14002504600F068F805460E4611
:10068000504659464246FFF771FF084305D0012006
:1006900004E020463946BDE8F08D0020054346EAD7
:1006A000E0762C4337430A986305E40AA0EB080080
:1006B0000022FD0A44EA47540A3002D500200146D0
:1006C000E9E7010510196941DDE9084500196941AB
:1006D000BDE8F04DA2E70EB5C10F80EAE070084416
:1006E000CA07002140F233438DE80E000A460B464C
:1006F000FFF7A3FF03B000BD30B5041E71F1000485
:1007000004DB4FF00044404264EB0101141E73F11E
:10071000000405DB1C464FF00043524263EB040328
:100720008B4208BF824230BD064C074D06E0E068B0
:1007300040F0010394E8070098471034AC42F6D328
:10074000FFF726FD2822000848220008202A04DBA3
:10075000203A21FA02F00021704721FA02F3D0403A
:10076000C2F1200291400843194670476FEA1121F7
:10077000016070470029816802D041F0010101E069
:1007800021F0010181607047084B10B5D3F80423B4
:1007900007490A40D0E900142143D0E9024004434C
:1007A00021431143C3F8041310BD00000020014091
:1007B000E030FCFF70B50D468EB01446012100F00C
:1007C00099FD0121080200F0ADFD03260B948DF880
:1007D000306000248DF833400BA9284600F0E8FB78
:1007E0004FF48030CDE90640089406A80994FFF73D
:1007F000CBFF0125E806CDE9024000948DF80440C6
:100800000494154C8DF805508DF814506946204617
:1008100000F04EF812208DF828008DF82960022093
:100820008DF82A008DF82B500AA800F0F1FC012267
:1008300040F20521204600F031F8062301220D2167
:10084000204600F05BF801212046FFF793FF204689
:1008500000F08EF80EB070BD00200140C06C80B278
:1008600070470246002012680A4200D001207047FB
:1008700010B5084C02212046FFF7F3FF20B12046B7
:10088000FFF7ECFF044908802046BDE81040022134
:10089000FFF76CBF002001400200002001238B40C5
:1008A00041680AB1194300E0994341607047000074
:1008B00030B542680F4B0C791A400B6842EA0422AB
:1008C0001343436082680C4B4D791A40D1E90343CE
:1008D00023438C6844EA4504234313438360C26A7C
:1008E000097D22F47002491EC9B242EA0151C16277
:1008F00030BD0000FFFEFFFCFDF7FFC070B507260E
:1009000009290AD9C568A1F10A0404EB4404A640E8
:10091000B543A3401D43C56007E0056901EB4104F1
:10092000A640B543A3401D4305611F23072A09D2F2
:10093000446B521E02EB820293409C4391400C4355
:10094000446370BD0D2A09D2046BD21F02EB8202F0
:1009500093409C4391400C43046370BDC46A0D3ABC
:1009600002EB820293409C4391400C43C46270BDF1
:10097000816841F080418160704700000EB5002021
:10098000029000F005FC02A9684600F01BF8094A35
:10099000029991420DD107280BD10749BDF80000FB
:1009A00008800649BDF8020008800549BDF804002A
:1009B00008800EBD0A554E011000002012000020D4
:1009C0000000002070B50F4E0D46044686B0002191
:1009D000304600F072F9002812D06A4600213046F5
:1009E00000F0D3F9019828600021684603E042181E
:1009F000D27A6254491C9DF80A208A42F7D8D0B2B4
:100A000006B070BD00640040F0B585B00023CDE9AC
:100A1000003104218DF808108DF809308DF80A2076
:100A2000694603E0C45CCD185B1CEC729342F9D3B9
:100A30000B4F384600F0F0F9064600244FF6FF75DC
:100A400000E0641C3146384600F038FA08B9AC4280
:100A5000F7D3AC4202D3012005B0F0BD0020FBE784
:100A60000064004038B50F4D09240B234FF4006299
:100A700029460120009400F083F80C23AA1429468B
:100A80000120009400F07CF801220221142000F0E3
:100A90006EF901B02802BDE83040034B034A044917
:100AA00000F016B9000002400A574E010A554E01E7
:100AB00000640040F0B5827A2F4D012191402A68F0
:100AC00042F001022A602C4E1C3632688A433260A2
:100AD000294A047B294B0C32A4B914688C43146056
:100AE0004488C78844EA0744877A03EBC707C7F8F6
:100AF00040460488878844EA0744877A03EBC7079F
:100B0000C7F84446047B012C12D114680C431460CE
:100B1000847A026803EBC4044FEA3242C4F84026E8
:100B2000847A426803EBC4034FEA3242C3F8442696
:100B3000114AC37A121D002B136806D00B431360B1
:100B40000D4A0389143213B104E08B43F7E71368AD
:100B50008B4313600389012B02D113680B4313608D
:100B6000407B012802D1306808433060286820F0BB
:100B700001002860F0BD00000066004000600040F9
:100B80002DE9FC410D461F4614460121089E00F048
:100B9000B1FB32463946284600F046FA02218DF86C
:100BA000041000218DF8061003208DF805000120A7
:100BB0008DF8070000946946284600F0F9F9BDE871
:100BC000FC81002A426901D00A4300E08A43426165
:100BD000704710B50368002223F002030360036826
:100BE00043F0010303604FF6FF7300E0521C4468BA
:100BF000E40701D19A42F9D14268D2073ED08A79FE
:100C0000012A02683CD022F080020260CA79012ADF
:100C1000026838D022F0400202600A7A012A026893
:100C200034D022F0200202604A7A012A026830D0D1
:100C300022F0100202608A7A012A02682CD022F087
:100C400008020260CA7A012A026828D022F004024F
:100C500002608A78CC78920742EA04620C7942EA10
:100C600004424C79098842EA0452491E0A43C2618F
:100C7000016821F001010160002114E0002010BD95
:100C800042F08002C1E742F04002C5E742F0200294
:100C9000C9E742F01002CDE742F00802D1E742F086
:100CA0000402D5E7491C4268D20701D09942F9D124
:100CB0004068C007E2D1012010BD0246002029B1E2
:100CC000012902D1106900F003007047D068FAE7EB
:100CD0002DE9F041884688B01E461746012100F0F4
:100CE00015FB00248DF806408DF8074007208DF88D
:100CF000040004208DF8084001258DF802408DF88D
:100D000005008DF809508DF8034006208DF80A4043
:100D1000ADF800008DF80B4069464046FFF759FFDB
:100D2000780BADF80C004FF6FF7000EAC701091D03
:100D3000ADF80E10710B00EAC6008DF81640ADF844
:100D40001010001D8DF817508DF81850ADF81200D6
:100D5000ADF814408DF8195003A8FFF7ABFE01223F
:100D600002214046FFF72DFF08B0BDE8F08108B52D
:100D70008DF800008DF801108DF8022001208DF80B
:100D80000300684600F044FA08BD10B500EB0113FB
:100D9000D3F8B04114F004041472D3F8B04133D046
:100DA000E4085460D3F8B04104F002045472D3F85C
:100DB000B44104F00F049472D3F8B441240AD474FB
:100DC000D3F8B841D472D3F8B841240A1473D3F8D5
:100DD000B841240C5473D3F8B841240E9473D3F85B
:100DE000BC41D473D3F8BC41240A1474D3F8BC4179
:100DF000240C5474D3F8BC311B0E937439B10169BF
:100E000041F02001016110BD640D1460CAE7C168A2
:100E100041F02001C16010BD30B50246002093684A
:100E20005B0108D49068000101D5012003E09068BF
:100E3000C00037D5022002EB0012D2F8803103F057
:100E40000103C2F880310B7A73B3D2F880414D6848
:100E50001C434B7A43EAC5031C43C2F880418B7A9A
:100E600003F00F038B72D2F8843123F00F03C2F822
:100E70008431D2F884318C7A2343C2F88431CB7A1E
:100E8000CC6843EA0423C2F88831CB7B096943EA82
:100E90000121C2F88C11D2F8801141F00101C2F891
:100EA000801130BD042030BDD2F880314C7A23430C
:100EB0000C8843EA4453C2F88031D0E7002221B1C4
:100EC000012905D0022906D112E08268114801E00B
:100ED0008268114802401149501A8A4214D00ADC33
:100EE000A2B16FF0806010180FD002280CD10FE073
:100EF00082680B48EEE7B0F5007F09D00949401839
:100F000003D0B0F5003F03D00020704702207047A7
:100F100001207047030000040003000800010008DE
:100F2000000003100001FFF770B505464FF6FF7093
:100F300000234AF201040DE0EA5C50400822C60793
:100F40004FEA500000D06040521E12F0FF02F6D16E
:100F50005B1C9BB28B42EFD370BD7CB50D46144633
:100F6000012100F0C7F901228DF8042000228DF83C
:100F7000062003208DF8050002208DF8070000945C
:100F80006946284600F014F87CBD7CB50D46144631
:100F9000012100F0AFF900228DF804208DF8062021
:100FA00000948DF807206946284600F001F87CBDC2
:100FB000F0B5002201274FF0030C0B6807FA02F589
:100FC0002B40AB422CD1066853000CFA03F4A64325
:100FD00006600E79D0F800E09E4046EA0E060660F4
:100FE0000E79012E01D0022E12D18668A6438660AA
:100FF0004E79D0F808E09E4046EA0E0686604668C4
:10100000AE43466045688E799640B6B2354345603A
:10101000C568A543C560CC799C40C3681C43C460C7
:10102000521C102AC9D3F0BD4B07DB0E9A40C908E9
:1010300010B500EB8100016A0F249C40A1430162BE
:10104000016A1143016210BD0246002012690A4282
:1010500000D0012070474183704701837047426987
:101060004A4042617047000010B52DED068B9FEDA0
:101070002D9AFFF73FFA9FED2C8B53EC182BFFF7BF
:1010800058F99FED2B1B53EC112BFFF7C4F9FFF719
:1010900051FA09EE900A19EE900AFFF738FA53EC6C
:1010A000182BFFF743F929EE290A41EC180B10EE33
:1010B000100AFFF72CFA53EC182BFFF7ACF9FFF7E7
:1010C00039FA00EE100A9FED1C8B9FED1DABC0EEB0
:1010D000090A10EE900AFFF71AFA41EC100B00F023
:1010E0003BFD53EC1A2B51EC100BFFF794F953EC2A
:1010F000182BFFF777F841EC100B53EC102B9FEDFA
:10110000120B51EC100BFFF786F99FED111B53ECFE
:10111000112BFFF708F9FFF70DFABDEC068B00EE77
:10112000100A10BD00401C466666666666660A4088
:101130000000000000FEAF40000000E0E1796B3FDE
:101140000000000000DCAE40000000000000F03FA6
:101150006666666666127140FEE770B504460D4627
:1011600045F2555000F02AF8204600F01BF82846BA
:1011700000F01EF800F00EF8BDE87040AFF30080FC
:1011800002494CF6CC400860704700000030004037
:10119000AFF3008002494AF6AA20086070470000B9
:1011A00000300040014948607047000000300040B6
:1011B0000149886070470000003000400149086024
:1011C0007047000000300040012202492020FFF754
:1011D000C4BE00000014024010B50C494FF0E023DB
:1011E00048689A694C68A042FAD1096801EB41034A
:1011F000C3EBC113C2EBC302B2FBF1F100EB40023F
:10120000C2EBC01001EBC00010BD000018000020B0
:1012100030B50F23C27801780125FAB1144A12685B
:1012200001F1E02102F4E062C2F5E062C2F30722BC
:10123000C2F10404D3404278A24084781C40144395
:10124000220181F80024007800F01F018D40400940
:10125000800000F1E020C0F8005130BD01F01F0017
:1012600085404809800000F1E020C0F8805130BD81
:101270000CED00E002490843024908607047000095
:101280000000FA050CED00E070B543F60342154985
:101290004020FFF77AFE4FF44044224612492020B6
:1012A000FFF773FE114D1F2229460820FFF755FE58
:1012B0000F4E4FF4704231460220FFF74EFE1B21C5
:1012C0002846FFF7CAFEA1103046FFF7C6FE2146AA
:1012D0003046FFF7C0FE2846BDE870400421FFF706
:1012E000BABE00000018024000140240000C024088
:1012F00000040240044A0029116801D0014300E0C3
:10130000814311607047000030380240044A0029D0
:10131000116801D0014300E0814311607047000073
:1013200040380240044A0029116801D0014300E01E
:1013300081431160704700004438024070B5204B73
:101340001968204C11F00C0104D06610042903D058
:10135000082903D004601BE0066019E0184A121F38
:101360001168C1F38055116801F03F0115B1B6FB5A
:10137000F1F101E0B4FBF1F114681268C4F38814D0
:101380006143C2F30142521C5200B1FBF2F1016011
:1013900019680F2202EA11110B4A545C0168E140FE
:1013A00041601C68072505EA9424145D21FA04F4C1
:1013B00084601B6805EA5333D25CD140C16070BDC4
:1013C000083802400024F40058000020174830B4C8
:1013D000018817480022B2EE040A0170090A417020
:1013E0001449441E097881701349C270D1ED000A76
:1013F00020EE800ABCEEC00A10EE101A017110EE49
:10140000101A090A41710F218171217801F1C0037D
:10141000C371491CC8B220701F2800D3227030BC91
:10142000082206490248FFF7EFBA0000100000202A
:1014300021000020000000200C00002001534E017C
:101440000CB50022274900920192086840F48030D0
:1014500008604FF4A043086800F400300190009841
:10146000401C0090019810B900989842F3D1086888
:10147000800334D5012001901A484030026842F0C0
:10148000805202601848026842F4404202601548E7
:10149000083002680260026842F40042026002689A
:1014A00042F4A0520260031F104A1A600A6842F018
:1014B00080720A600A689201FCD50D4940F20572FB
:1014C0000A60016821F003010160016841F0020136
:1014D00001600168C1F381010229FAD10CBD0192BA
:1014E0000CBD000000380240007000400854400766
:1014F000003C0240094810B50168094C6268891A2D
:1015000064290AD3006860606088FFF7ADFD84ED50
:10151000030ABDE81040FFF759BF10BD1C000020B2
:10152000000000200E4810B501680E4CA268891A10
:10153000B1F5FA7F13D30068A06001210A48FFF7D4
:101540008EFD228809484FF4804112B1FFF785FDD6
:1015500001E0FFF780FDBDE8104000F003BE10BDC4
:101560001C00002000000020001402400004024083
:101570002DE9F05F61480168491C0160604F4FF43C
:1015800000613846FFF760FD5E4EDFF87CB15F4CCE
:10159000002558B12068401C206003280DDD04217F
:1015A0005846FFF758FD0120307006E0256030787E
:1015B00018B904215846FFF750FD01213846FFF7BE
:1015C00043FDDFF84CA14FF4004628B16068401C91
:1015D0006060032809DC0CE04E486560008820B19B
:1015E00031465046FFF739FD03E031465046FFF7DC
:1015F00032FD02213846FFF727FD4FF4804928B11C
:10160000A068401CA060032809DC0CE04248A560EB
:10161000008820B149465046FFF71FFD03E04946C8
:101620005046FFF718FD4FF480613846FFF70CFD78
:1016300048B1E068401CE060032805DD02215846FF
:10164000FFF709FD00E0E5604FF400713846FFF751
:10165000FBFC48B12069401C2061032805DD012105
:101660005846FFF7F8FC00E0256131462B4E304626
:10167000FFF7EAFC4FF4805848B16069401C606194
:10168000032805DD41465046FFF7E5FC00E06561B3
:1016900049463046FFF7D8FC4FF4005648B1A069E0
:1016A000401CA061032805DD31465046FFF7D3FCFE
:1016B00000E0A56141463846FFF7C6FC48B1E06945
:1016C000401CE061032805DD08215846FFF7C3FCF4
:1016D00000E0E56131463846FFF7B6FC50B1206ABC
:1016E000401C2062032806DD5846BDE8F05F10214B
:1016F000FFF7B1BC2562BDE8F09F00001C00002090
:101700000018024014000020000C02402C000020B1
:1017100000040240100000200000002000140240DD
:10172000124810B5016841F4700101601048016869
:1017300041F0010101600E4A002108321160026887
:101740000C4B1A400260031D0B4A1A60026822F417
:101750008022026006480C300160FFF771FE0349E9
:101760004FF000608039086010BD000088ED00E097
:1017700000380240FFFFF6FE1030002410B5074C81
:101780000121204600F00FF8002805D02046BDE8D2
:101790001040012100F004B810BD0000000001401D
:1017A000C9430182704702460020138A92890B4286
:1017B00002EA010202D0002A00D001207047000096
:1017C00070B5104D40F225542146284600F0C5F86A
:1017D00050B1284600F086F90B4A2146906228460F
:1017E000BDE8704000F036B840F224412C4628464F
:1017F00000F0B3F8002803D020880248001D0088BC
:1018000070BD0000004C00402C00002070B50F4D52
:1018100040F225542146284600F09FF850B1284652
:1018200000F060F90A4A214650622846BDE870403F
:1018300000F010B840F224412C46284600F08DF804
:10184000002801D02088A08870BD00000010014051
:101850002C0000200A0A01219140C94301807047F1
:101860000029818902D041F4005101E021F40051A6
:1018700081817047F8B509201E4D00904FF4007328
:101880002A460721012000F041F80A242E1533468C
:101890002A4607210120009400F038F80022032195
:1018A000252000F011F94FF416552B46124A10214D
:1018B000124800F0DFF80094114C3346224608210C
:1018C000042000F023F80B200090E31422460821A6
:1018D000042000F01BF800220321342000F0F4F86B
:1018E00001B02B467102BDE8F040064A064800F000
:1018F000C1B800000000024000100140251300089C
:1019000000080240004C00400D1300082DE9FC4186
:101910000E461C4615460121089FFFF7EBFC324698
:1019200039462846FFF780FB02218DF804108DF818
:10193000051000208DF8060001208DF807000094A6
:1019400069462846FFF734FBBDE8FC8102460020CB
:1019500012880A4200D00120704770B501F01F05BF
:1019600001260024C1F3421306FA05F2012B0FD021
:10197000022B0FD0838A4FEA11210088134206FA06
:1019800001F600EA060001D000B10124204670BD36
:101990008389F0E7038AEEE710B5C1F3421301F043
:1019A0001F040121A140012B07D0022B07D01430C6
:1019B000002A026805D00A4304E00C30F8E7103032
:1019C000F6E78A43026010BD7FB50446008A0D46E3
:1019D000C98820F4405001432182A08941F20C6162
:1019E0008843A9882A8911436A8902431143A18146
:1019F000A08A20F44071A8890843A0826846FFF7B6
:101A00009DFC1A48844202D01948844201D10398AF
:101A100000E00298A189090400EBC00101EB00106D
:101A2000296801D5490000E08900B0FBF1F064228B
:101A3000B0FBF2F109010B096FF018056B4300EBE5
:101A40008300A3891D044FF0320306D503EBC000C9
:101A5000B0FBF2F000F0070005E003EB0010B0FB74
:101A6000F2F000F00F00084320817FBD001001401C
:101A7000001401407FB516460A4605461C46012162
:101A80001046A8470020ADF80800ADF804000C216E
:101A9000ADF80600ADF80A10ADF80C0000946946E8
:101AA0003046FFF791FF012240F225513046FFF703
:101AB00073FF012240F224413046FFF76DFF012100
:101AC0003046FFF7CDFE7FBD08B58DF800008DF8DC
:101AD00001108DF8022001208DF803006846FFF701
:101AE00097FB08BD8088C0F308007047C1F3080168
:101AF0008180704770B506460024FFF7F7FF4CF26F
:101B0000503502E0641CAC4205D880213046FFF716
:101B10001DFF0028F6D070BD2DE9F04100251646C6
:101B20000F4680462C4605E0395D4046FFF7E2FF50
:101B3000641CE4B2B442F7D34CF250344021404626
:101B4000FFF704FF002803D16D1CADB2A542F5D903
:101B5000BDE8F0810000000070B5D94B00242DEDE8
:101B6000020B2DED108BDDE91010984205DA20F004
:101B700000429A4201D809D141B19DED100BBDEC54
:101B8000108B02B0BDE8704000F05EBAB0F5801F67
:101B900026DA11430BD0002813DA012000F080FA76
:101BA000BDEC108B02B0BDE8704000F059BA0220C5
:101BB00000F076FA00F030FA51EC100B81F00041A1
:101BC0009EE06FF035049FEDC00B53EC102B9DEDA4
:101BD000100B51EC100BFEF7ACFBCDE910010846E1
:101BE00004EB2051C0F31304B948A1F2FF312044A3
:101BF00000F4801080F07F6282F04052224301EBBB
:101C000020559FEDB50B119253EC102B9DED100B51
:101C100051EC100BFEF787FB41EC180BA01CC0F336
:101C200013009FEDAFDB9FEDB0EBB14E7E44032878
:101C30006CD296ED000B51EC180B53EC102BFEF709
:101C40005BFD1DD1002D01BF96ED000BBDEC108B8F
:101C500002B070BD2846FEF73EFD41EC180B53EC78
:101C60001D2BFEF766FB41EC190B53EC1E2B51ECC0
:101C7000180BFEF75EFB53EC192BFEF7B3FA3FE0AF
:101C80009FED9D0B51EC180B53EC102BFEF751FB05
:101C90009FED9B1B53EC112BFEF748FB41EC190BFE
:101CA00053EC182B51EC180BFEF743FB53EC192B9C
:101CB000FEF73FFB41EC190B002D04BF53EC192B31
:101CC00051EC180B1AD02846FEF705FD41EC1A0B13
:101CD00053EC1D2BFEF72DFB53EC192BFEF726FBC7
:101CE00053EC182BFEF71FFB41EC180B53EC1E2B8B
:101CF00051EC1A0BFEF71DFB53EC182BFEF713FBF0
:101D0000BDEC108B02B041EC100B70BD9FED7E0B53
:101D100051EC180B53EC102BFEF764FA41EC100B4E
:101D200051EC180B53EC102BFEF775FB41EC190B23
:101D30002846FEF7D0FC41EC1B0B53EC192B51EC61
:101D4000190BFEF7F6FA41EC1A0B714853EC1A2BFB
:101D5000261851EC1A0BFEF7ECFA41EC1F0B6D48FC
:101D6000C4F1510404F5D724B0EE4F0AF0EE6F0A27
:101D70000321784400F0D2F853EC1F2B51EC100BE8
:101D8000FEF7D7FA41EC1C0B6348B0EE4F0AF0EEB9
:101D90006F0A0421784400F0C1F853EC1A2B51EC7F
:101DA000100BFEF7C6FA344353EC1C2BFEF71AFA5D
:101DB00041EC1C0B002C4CDD9FED510B51EC180B32
:101DC00053EC102BFEF7B5FA53EC182BFEF7B1FAD3
:101DD00041EC1A0B55B353EC1D2B51EC1B0BFEF7CA
:101DE000A8FA41EC1D0B53EC1C2B51EC1A0BFEF71F
:101DF000F9F953EC192BFEF79CFA53EC1D2BFEF767
:101E0000F1F953EC1A2BFEF791FA53EC182BFEF76D
:101E10008AFA41EC180B53EC1E2B51EC1B0BFEF70E
:101E200088FA53EC182BFEF77EFA69E753EC1C2B6B
:101E300051EC1A0BFEF7D6F953EC192BFEF779FA91
:101E400053EC1A2BFEF772FA53EC182BFEF76EFACE
:101E500056E735B353EC1D2B51EC1B0BFEF769FA1B
:101E600041EC1A0B53EC1C2B51EC180BFEF75BFAF0
:101E700053EC192BFEF75DFA53EC1A2BFEF753FACD
:101E800053EC182BFEF74FFA41EC180B53EC1E2BBA
:101E900051EC1B0BFEF74DFA53EC182BFEF743FAEF
:101EA0002EE753EC1C2B51EC180BFEF73CFA53ECCD
:101EB000192BFEF73EFA53EC182BFEF737FA1FE703
:101EC0000000F07F00000000000000000000504310
:101ED000645F090000000000000000000000F03F07
:101EE000763C7935EF39EA3D0000E0FE422EE63FD0
:101EF000F005000000000000555555555555D53FDB
:101F0000000000000000E03F000000000000004072
:101F100086EBF9FF720400006804000070B5044607
:101F20002DED028B4D1E00EBC500B0EE408AF0EEA9
:101F3000608A90ED000B35F0060017D053EC182B9B
:101F400051EC100BFEF7F5F941EC100B6D1E04EB94
:101F5000C50090ED001B51EC100B53EC112BFEF75C
:101F600041F941EC100B35F00600E7D1022D36D0D7
:101F7000042D1CD0062D1CBFBDEC028B70BD53EC94
:101F8000182B51EC100BFEF7D4F994ED0A1B53EC0F
:101F9000112BFEF727F953EC182BFEF7CAF994ED35
:101FA000081B53EC112BFEF71DF941EC100B53EC01
:101FB000182B51EC100BFEF7BCF994ED061B53ECFB
:101FC000112BFEF70FF953EC182BFEF7B2F994ED35
:101FD000040B53EC102BFEF705F941EC100B53ECFE
:101FE000182B51EC100BFEF7A4F994ED021B53ECE7
:101FF000112BFEF7F7F853EC182BFEF79AF994ED36
:10200000001B53EC112BFEF7EDF8BDEC028B41ECFD
:10201000100B70BD000000009FED070B10B553ECD6
:10202000102B9FED070B51EC100BFEF7F4F941EC70
:10203000100B10BD000000000000000000000000B8
:10204000000000000000F03F10B553EC102B51ECE5
:10205000100BFEF7C7F841EC100B10BD000000009C
:102060009FED050B10B553EC102B51EC100BFEF748
:10207000D2F941EC100B10BD000000000000000080
:1020800002E008C8121F08C1002AFAD17047704741
:10209000002001E001C1121F002AFBD1704700009F
:1020A0000149086070470000680000201FB56846BD
:1020B000FFF744F90D490098B0FBF1F00C490860B6
:1020C00001984FF47A71B0FBF1F0401EB0F1807FBF
:1020D0000AD24FF0E0214861064AF02082F8140D40
:1020E00000208861072008611FBD000040420F00EA
:1020F000180000200FE000E030B50446FFF76CF850
:10210000054604EB4400C0EBC414FFF765F8401B20
:10211000B0EBC40FF9D330BD4FF4A060FFF7AAF8BD
:10212000FFF7C4FF08220E490420FEF743FBFEF729
:1021300099FCFFF79FFBFFF747F8FFF7A5F840F67C
:10214000B830FFF7D9FF4FF47A710420FFF705F894
:10215000FFF71EF8FFF7CEF9FFF7E4F9F8E7000004
:102160000008024000B587B01C2214A16846FEF7A3
:1021700027F81948018819480129008800D018B1AA
:1021800001218DF80C1002E000208DF80C008DF874
:102190000E0019216846FEF7C7FE8DF81900000AE7
:1021A0008DF81A001B2269460D48FFF7B5FC1B226B
:1021B00069460C48FFF7B0FC07B000BD01100100F4
:1021C00000091200030000000000000000000000F1
:1021D000010001000100000010000020120000209A
:1021E00000100140004C004004FA97999999D93F9A
:1021F000AF788E1DC571CC3F9FC678D0099AC33F7A
:10220000935555555555E53F599322942449D23F4E
:10221000DE03CB966446C73F44523EDF12F1C23F15
:10222000000000000000000048220008000000201C
:102230006C00000080200008B42200086C00002020
:1022400004040000902000080000000000000000CE
:10225000000000000000000000000000000000007E
:10226000000000000000000000000000000000006E
:10227000000000000000000000000000000000005E
:10228000000000000000000000000000000000004E
:10229000000000000000000000000000000000003E
:1022A00000000000010203040102030406070809FC
:0422B000000000002A
:040000050800018965
:00000001FF
